:100000006F20005600000000162200001822000099
:1000100000000000000000000000000000000000E0
:1000200000000000000000000000000000000000D0
:100030001A2200000000000030250000000000002F
:100040003225000034250000362500003825000048
:100050003A2500003C2500003E2500004025000018
:1000600042250000442500004625000048250000E8
:100070004A2500004C2500004E25000050250000B8
:100080005225000054250000562500005825000088
:100090005A2500005C2500005E25000000000000DD
:1000A000511126C022C206C4828282441244A24058
:1000B000310182802A86014593F6150091C232955E
:1000C00085810606F5F9828000000000634E050276
:1000D00063C305042E86AA857D5515C285466378BF
:1000E000B6006356C00006068606E36CB6FE014500
:1000F00063E4C500918D558D85820582F5FA828075
:100100008682C93F2E8582823305A04063D70500D1
:10011000B305B040C1B7B305B0408682653F330533
:10012000A0408282868263C70500634905005D376F
:100130002E858282B305B040E35B05FE3305A04007
:10014000513F3305B04082820000EFF27FF52E86EA
:100150009305100AEF00D02E89BFEFF27FF47111E2
:100160002A84AE8432C0B7170140214798CB1306CA
:10017000E00A9305000AEF00B02C26869305000ADA
:100180002285EF00F02B82452285C137110131BF56
:1001900011CEEFF2FFF0C14763F3C7004146B286CC
:1001A0002E8693050009EF00B01001B78280EFF2B0
:1001B0003FEF91E18545FD1593F5F50F920593F518
:1001C000F50F850593F5F50FEF00900EF9BDEFF2F1
:1001D0003FED1301C1FD02C602C802CA02CC02CE25
:1001E00002D002C002C202C41165EF205011A14723
:1001F0007C8002C48A853715014013050540EF2035
:1002000060653724014013050440EF20A03D02C67D
:1002100002C802CAB7070E003ECC02CE85472300B3
:10022000F1026C0013050440EF20203E9D46054678
:10023000914513050440EF20204899460546814525
:1002400013050440EF20A054B70500021305044035
:10025000EF20605E854513050440EF20E03F130565
:100260000440EF20A0403725014013050540EF2052
:10027000804075F93725014013050540EF20804087
:100280003725014013050540EF20604075F9130143
:10029000410221BD814681473D476361F7021396C4
:1002A0001700370700201307470532971A23BA961D
:1002B000C206C182850793F7F70FF9BF9182B7078E
:1002C00000202398D7048280EFF29FDD85453725F3
:1002D000014013050540EF20603CC1BBEFF25FDC3D
:1002E00089453725014013050540EF20E05311E112
:1002F0006DBB138441820620938714001EA037250E
:10030000014013050540EF20A0468604B7070020F2
:1003100093874705A6978AA31E20BD8B1EA0A1C365
:10032000B727014093870740DC4393F70740E9D3A1
:1003300091453725014013050540EF20E04E4DD98A
:10034000D1453724014013050440EF20204C23936E
:10035000A182814513050440EF20004251BF1D3F9B
:10036000C1B7EFF2FFD3B707002003D50705930706
:10037000700263F5A700130585FD11A001459305E3
:10038000803D2A05813B09811345F5FF1375F50F63
:1003900029BBB7170140370710001307070298CB96
:1003A0009843B70601FFFD16758F98C39843B706AB
:1003B0008800558F98C3814731A893962700BE9631
:1003C00013962600138781823297914614A38507DE
:1003D00093F7F70F0547E372F7FE9387818255473E
:1003E00098B31147D8BBB71701409C4793F7070252
:1003F00099E79387818298231367870098A3828067
:10040000EFF21FCA01445DA0014799C3C18A99C296
:1004100063000718139724002697931627009387E5
:100420008182B697BA23C167FD17630CF7009396D4
:100430002400A6961396260093878182B29705071B
:10044000BAA31397240026979316270093878182D7
:10045000B697B623954763F8D704139724002697D9
:100460001316270093878182B297982393771700FA
:10047000C9E393878182B29713E7150098A39C473D
:100480009DC395E1228582979387818213972400EB
:1004900033069700931626003686BE96B2849C22B9
:1004A00093E707019CA205041374F40F854763E7E3
:1004B0008712A2841317240022979316270093878C
:1004C0008182B697902393758600371701401847AD
:1004D000943313F5F6008547B397A70093F7F70F0A
:1004E000F98F9DF313F7060119E33E8739BF0547DE
:1004F00029BF139624002696131526009387818220
:10050000AA97DE23E3E1F6FA9377270091C7938752
:100510008182AA97FE23C1DB93962400A6961396A8
:10052000260093878182B2971367270098A3DC4740
:1005300085C399ED228582971397240026979316F9
:10054000270093878182B69798231367070298A3A1
:100550001397240026979316270036879387818266
:10056000B697F623BE2363F9D700BA8493878182B6
:10057000BA972391070005BF13972400BA941396E6
:100580002400B284138781823297958F3EA321BFC6
:10059000118AE31A06F01397240026979316270072
:1005A00093878182B697114798A3239107009C4BAC
:1005B000E38B07EEE39905EE22858297938781828C
:1005C0001397240033069700931626003686BE96AE
:1005D000B2849C2293E707049CA2F1B5F9B4138777
:1005E000018501458147B54663EBF6001423369536
:1005F000420541818507C207C1830507EDB78280A7
:10060000EFF21FAA2A8493840185D14613860185BF
:10061000814501455128E1379848B7E72420938761
:1006200027C36304F7041384018523000400914762
:100630001CB0A301040089475CA0E5475CB0A1475A
:100640007CA0930700FC7CB09307F0071CA499479B
:100650001CB495473CA4D1573CB451376AA4B7E7C2
:100660002420938727C31CC889B493870185FE275C
:10067000E39BA7FA75D845BFEFF29FA28D3713848D
:1006800001856AA4B7E72420938727C31CC8C14605
:1006900013860185814501450520C14613060401E5
:1006A000C1450145112811B4EFF29F9F0605398914
:1006B0001365050AE522D5BAEFF29F9E61112EC09F
:1006C00032C2B6841314150039881364040AB7E7DC
:1006D00000E0056723A0E718B717014013070004DF
:1006E000D8CB22858D2B75DDA686124682452285C4
:1006F000C12622858D2375DDB7170140130700043D
:1007000098CBB7F700E023A4070023A20700B7E7C0
:1007100000E0056723A0E710210141BAEFF25F98DE
:1007200031112AC42EC6B28436C03AC2C5CD224782
:10073000135487401374F40F1547637387001544EF
:100740001377240001E73E8782473AC013774400BD
:1007500009E70247924636C03AC21377640059EB64
:100760001377140001C702473EC0BA8784A3B2477B
:1007700093C5F7FF1395040141812AC893F5F50F3E
:10078000EFF05F9342054181930715001395070130
:10079000418193578500AA97C207C183A18312475D
:1007A0001CA30C84058825E8A9EDB24713958700A2
:1007B00093558500AA95C205C181A18193C5F5FF16
:1007C00093F5F50F4245EFF0FF8E4205418193D737
:1007D000140093F7F70F3E9542054181218182472E
:1007E00088A331A090A3924790A3B68790A351010C
:1007F0006FF0BF8B1377140035FB02473EC0BA87FA
:10080000B5B7B305B04093F5F50F3245EFF09F8AC9
:100810004205418171BF0C843245EFF0BF899315C9
:100820000501C18193D78500BE95C205C181A18113
:1008300093C5F5FF93F5F50F4245EFF0BF874205ED
:10084000418193D7140093F7F70FAA97C207C1838A
:10085000A18302471CA361BFEFF29F84411102C232
:1008600002C402C6B7370A009387A7C23EC0F17719
:10087000FD177C83930700407C8591677C868A8581
:100880003754004013050440EF20E0098545130567
:100890000440EF20601741016FF03F81EFF25F806D
:1008A00061112AC02EC2B2843684C167FD1723A20B
:1008B000F186B70502003755004013050540EF20CB
:1008C000E01F01C99387418698439306F7FF94C3BD
:1008D0006DF383A741866383071C85453755004028
:1008E00013050540EF200014C167FD1723A2F18610
:1008F000B705030085053755004013050540EF2077
:10090000001A01E99387418698439306F7FF94C341
:1009100065F383A7418663850718014682453755ED
:10092000004013050540EF204016C167FD1723A2C4
:10093000F186B70507009385250837550040130554
:100940000540EF20C01501E993874186984393063F
:10095000F7FF94C379FF83A7418663850714814518
:10096000B757004013850740EF20800F9245B757D7
:10097000004013850740EF208010C167FD1723A2B8
:10098000F186B705070093854508375500401305E4
:100990000540EF20C01001E99387418698439306F4
:1009A000F7FF94C379FF83A74186638F070E8545C0
:1009B000B757004013850740EF20800A8545B75799
:1009C000004013850740EF20E005C167FD1723A213
:1009D000F186B7050300850537550040130505402E
:1009E000EF20E00B01E99387418698439306F7FFD8
:1009F00094C365F383A74186D5CB05468245375519
:100A0000004013050540EF204008C167FD1723A2F1
:100A1000F186B705030089053755004013050540E9
:100A2000EF20E00701E99387418698439306F7FF9B
:100A300094C365F383A7418695E36955A9A8938775
:100A400014003EC03755004013050540EF206003F9
:100A500088A07D141374F40F15C4824405CCB70527
:100A60000010938505043755004013050540EF201D
:100A7000E00471F5A2853755004013050540EF10DD
:100A8000307EF1BF85453755004013050540EF1016
:100A9000507BE1B7014521016FF02FE17D55E5BFA6
:100AA0007955D5BF7555C5BF7155F5B76D55E5B7C6
:100AB000EFF20FDF51112AC22EC432C03684C16753
:100AC000FD1723A2F186B705020037550040130534
:100AD0000540EF10B07E01C9938741869843930685
:100AE000F7FF94C36DF383A741866385071485459B
:100AF000B754004013850440EF1090768545138568
:100B00000440EF103072C167FD1723A2F186B705CC
:100B1000030085053755004013050540EF10307878
:100B200001E99387418698439306F7FF94C365F3E1
:100B300083A74186638207100146924537550040DE
:100B400013050540EF107074C167FD1723A2F186ED
:100B5000B705070093852508375500401305054064
:100B6000EF10F07301E99387418698439306F7FFEE
:100B700094C379FF83A74186F1C3A245375500404E
:100B800013050540EF10B06FC167FD1723A2F18672
:100B9000B705070093854508375500401305054004
:100BA000EF10F06F01E99387418698439306F7FFB2
:100BB00094C379FF83A7418685EF71558DA882473D
:100BC000938417008C233755004013050540EF1020
:100BD000106B7D141374F40FB70507009385450857
:100BE0003755004013050540EF10706B75D526C0D2
:100BF0001DC4B7050010938505083755004013053F
:100C00000540EF10B06B45FDB7050010938505401A
:100C10003755004013050540EF10506A71D98545DE
:100C20003755004013050540EF10B0610145310113
:100C30006FF0AFC77D55E5BF7955D5BF7555C5BFB9
:100C4000EFF20FC67111D0818546130631008D3544
:100C500011016FF08FC5EFF2AFC493574500638663
:100C600007109377850F1307800F6384E7102A849A
:100C7000C167FD1723A2F186B70502003755004072
:100C800013050540EF10906301C99387418698438F
:100C90009306F7FF94C36DF383A74186638D070C1A
:100CA00085453755004013050540EF10B057C16723
:100CB000FD1723A2F186B7050300850537550040CF
:100CC00013050540EF10B05D01E993874186984315
:100CD0009306F7FF94C365F383A74186C5C3937456
:100CE00014002686A2853755004013050540EF10F5
:100CF000D0591307001823A2E186A9E0B704070022
:100D000093842408A6853755004013050540EF104D
:100D100010591DC99387418698439306F7FF94C3E2
:100D200015C3B705001093850540375500401305DE
:100D30000540EF10B05879D5814401A8B7040300ED
:100D40008904C9B7854411A0854483A7418691E3EE
:100D500081443755004013050540231A0500854599
:100D6000EF10304E81C4A28411A0814426856FF01B
:100D7000CFB38144E5BF9304F00FCDBF9304E00FE0
:100D8000F5B7EFF2EFB1411102C002C202C423165F
:100D9000010023070100FD575C8081472DA01387C8
:100DA000C18693961700B385F60013961500B28599
:100DB0003A9623100600231106002E9723120700EF
:100DC000850793F7F70F2147E37BF7FC938781862D
:100DD00023810700A38007002380070001469305B5
:100DE000100713058006EFF04FB781473947636B53
:100DF000F70018083E97FD562308D7FE850793F79E
:100E0000F70FEDB73D468A8513058006EFF04FB822
:100E100041016FF08FA90547A385E186828083C7D2
:100E2000B186D1E782808D67938747D4BA979C2398
:100E3000FD17FD8B9386C186131617003305E60058
:100E400093151500B69503D3050008103E952300B1
:100E500065FEAA2193851700130301029A9523804A
:100E6000A5FE3A9693151600AE96D62289079A9754
:100E70002380D7FE05071377F70FA147E3F5E7FABD
:100E8000938781869823230BE1009833A30BE1001D
:100E9000BC23230CF100FD460A8685451305800618
:100EA000EFF0EFB0A385018605616FF00FA0EFF2C0
:100EB0002F9F01110147D1B78D67938747C43E9596
:100EC00008218280858991E18280EFF26F9D411136
:100ED0002AC691371387018540231D889317240064
:100EE000B38687008D67938747D5B697BC239D8BC4
:100EF0003EC25C331397270093070060998FC207A7
:100F0000C1833EC485473EC081445DA81D8B638379
:100F1000E404138717001377F70F15456309A70833
:100F2000850693F6F60FBA8721476367D70813D76C
:100F300017001375F70F13172400330387000D678D
:100F4000130747D51A972A97182313F517005DFD45
:100F500011836DBF01CEA1CA1377F60039E711479F
:100F60006364D700814575B7854511A0DDD1138530
:100F7000018B8343050013971600B302D700139328
:100F800012009382C18616932310730083431500C9
:100F90002311730003432500369713151700AA92F7
:100FA00023926200BDB78545D9B781459DB71387A8
:100FB00027001377F70FADB72EC0850493F4F40F15
:100FC000924763E19704A6852245EFF0AF8E83D761
:100FD000418B930500603E95EFF0CF941387018B12
:100FE0009307270005079386018B1306F00F9305DF
:100FF000F00F42054185EFF06FF28147814682454F
:1010000032461DB71384418B0A2009059305006001
:1010100042054181EFF0CF8E0AA041016FF0EF88C9
:10102000EFF20F882A84138701857C33642313072A
:10103000D00F6361F7049305F00F1387018B1396AC
:101040001700B2971395170093072700050793869B
:10105000018B1306F00F42054185EFF02FEC93074B
:10106000D00F63EB970093D52400850593F5F50F1A
:1010700081470DA88145D1B79305F00FFDB71377D0
:10108000F4008546631DD7003E861387418A3E974C
:101090001423BDCE1387418A3E97FD1614A38507FE
:1010A000C207C18321476367F70679DC1147E3680C
:1010B000F7FC0547E38AE7FCDDB713171600329704
:1010C000369706071385C1862A97231007008506E1
:1010D000C206C1820947E364D7FC13171600329792
:1010E000369706071385C1862A970A2313930501AD
:1010F00013530301E373A3FC1317160032973697BB
:1011000006079382C1861697330565400AA3C1B7C7
:101110008146C9B783D7E18A6399070C03C6218A40
:1011200059E211C403C7318A8547631CF70283C69D
:10113000318A914763E7D7021387018B0823939580
:101140001600B695939715009385C186AE978AA32E
:101150000C33AEA33823DAA39387418AB697294785
:1011600098A309C43D8885476314F40483C7318A72
:101170000D47636FF702938557001387018B082390
:1011800093961500AE96939716009386C186B697F0
:101190008AA31433B6A33823DAA39387418AAE9780
:1011A000294798A331A083C7318A05476376F7049E
:1011B0001387318A1C23850793F7F70F1CA355C2A9
:1011C00009476378F700A381018A0506058A238110
:1011D000C18A83C7218AC1CB930680022397D18A13
:1011E00083C7318A6383E7083D319387E18A9A2375
:1011F0007D179AA36FE07FEB99E70DC08945054401
:101200004204418089A809CC3D8885476305F400E4
:10121000A5452544F5B7A5451544DDB79545CDB79A
:10122000A5451544F1BF1387018B082393161400BD
:10123000A296939716009386C186B6978AA3143315
:10124000B6A33823DAA39387418AA297294798A3A4
:1012500005044204418093970501C183E365F4FCD2
:1012600081BF1547B9BFD14695BF13070014239717
:10127000E18A9DBFEFE2DFE251112A842AC213877F
:1012800001853C3713961700B297139517009317F3
:101290000501C1833EC03C27BD8B93F7F70F139721
:1012A0001700BA971397570093170701C1833EC4DD
:1012B00083C701850D476383E70001C89581858950
:1012C0006391051081440144BDA013878186BA97BC
:1012D0008423F5D88544C5BF9386018B8822139754
:1012E0001700B305F700139615009385C1862E9657
:1012F0000AA288322AA2B0223E9793161700AE9611
:10130000D2A2850793F7F70F2147E377F7FC39A8B7
:101310009547DDBF9247ADCB1387018B142393878D
:10132000C186B6AB1433D6AB3823FAAB85048588B7
:1013300005041374F40F854763E787081387018B4F
:101340009307270005079386018B1306F00F93057B
:10135000F00F03150100EFF06FBC82472247338581
:10136000E7009305006042054181EFE07FD99317C4
:101370000501C1833EC0D9DC9247D9DBBD8B0D4747
:10138000E396E7FA954749B792471147E360F7FAC2
:101390009386018B882213971700B305F7001396E5
:1013A00015009385C1862E960AA288322AA2B02201
:1013B0003E9793161700AE96D2A2850793F7F70FC4
:1013C000E9B7854409B731016FE03FCE8D8991C1FE
:1013D0008280EFE2FFCCAA841385818C992D13754E
:1013E000F50F99C493F7F40009476383E700098177
:1013F000938701859C376364F5000144EDA813854C
:10140000818C052D4205418193171500AA971395EC
:1014100097004181938701858C2793978501E18708
:1014200063CF070686051387018B930727000507FF
:101430009386018B1306F00F93F5E50FEFF00FAED7
:101440001385818CFD2305647D14698C9305701CC4
:101450002285EFE03FC891CC8947630CF50093F7F4
:10146000F4000947E39BE7F885679387278EE3F647
:1014700087F81387018B102393161500AA9693976C
:1014800016009386C186B69792A31433B6A3382369
:10149000DAA39387818BAA970D4798A3B9BFB305A9
:1014A000B04093F5F50FBDBF1397160036973E97E2
:1014B00006071386C18632971223058212A3850779
:1014C00093F7F70F09476363F7021387818B36970A
:1014D000182379DB1397160036973E970607138675
:1014E000C186329712237D1612A3D1BFEFF0BF92AF
:1014F00005041374F40FA14763EB870281CC89477D
:10150000630AF40093F7F4000947E391E7FE91477B
:10151000E3FE87FCA2869387818BA2979C2391C7C9
:101520001387818B2297FD171CA3814761BF6FE052
:10153000DFB7EFE2FFB651112A8483C401858D47DE
:10154000638FF40283C7518C8DEF1387618C1C234A
:101550008507858B1CA3938701859C3386070D67C0
:10156000130787D8BA979A23A382E18C85473EC296
:101570009387518C98237D1798A3014729AA854406
:10158000D1B702C2F5B703C6618C31CE01CC91460A
:10159000630AD7009376F40011466398C602914619
:1015A00063F5E60293961400338696008D66938663
:1015B000C6D7B296BE968C2293161700BA96BE96E0
:1015C00086061386C186B2968EA2850793F7F70F1B
:1015D000894663EFF60AB706002083C64601E36733
:1015E000D7FAE382E6FA63FDE60201CC9146630A8C
:1015F000D7009376F4001146E399C6FC9146E3F6D2
:10160000E6FC8D66938606D5BE968C22931617004F
:10161000BA96BE9686061386C186B2968EA275B716
:1016200001CC1146630AC7001376F4009145E31E0E
:10163000B6F81146E37BE6F8E399E6F883C6618CD9
:10164000C9F693161700BA96BE9686061386C1860B
:10165000B29692229306000263FFC600931617000B
:10166000BA96BE9686069385C186AE96011692A25C
:10167000854636C299BF93161700BA96BE9686065F
:101680001386C186B29623900600854636C235BFC2
:1016900005071377F70FA14763E4E70081470DBF04
:1016A00069C0B707002083C64701A947638FF60AC0
:1016B00083D7218C639B071A370700201307470144
:1016C0001C23850793F7F70F1CA309C80D47636711
:1016D000F700B70700201147238AE700B70700206B
:1016E00083C747012547638CE71429476399E718A7
:1016F0001307401F2391E18CB9A293878186BA9783
:101700002380070005071377F70F8947E3F7E7FE04
:10171000B707002083C64701A147E3F4D7F883C782
:10172000618CB1C39306000F93878186A69794A31B
:1017300083C7518CA145E3E6F5F6B387F540B3D7EF
:10174000F64093F7F70F93868186A6969CA2AD4646
:10175000E3E9F6F4938781863386F40023000600DC
:1017600089B722875DB7B146C1B783C7418C894627
:1017700063F3F602FD172382F18C3DC091476303AA
:10178000F7069377F40091466395D704914763F287
:10179000E70402C01DA82382018CC5B782471387C6
:1017A000870106079387C1863E9783C5418C3AC45B
:1017B0000A23EFE03F9042054181218122470AA39D
:1017C0008247850793F7F70F3EC089470247E3F743
:1017D000E7FC9377F40011476381E70681471DA872
:1017E00022C0E5B702C0D5B71387C1860A3B9396DE
:1017F0001700B385F600139615003A960AA22E3B01
:101800002EA24E3BBE961396160032974EA3850726
:1018100093F7F70F1D47E379F7FCE31B04E8938781
:101820008186BE9483C5418C8820EFE0BF889317E2
:101830000501C183A1839CA0A5BD9547E1BF130706
:10184000803E2391E18CB707002003C74701A947D9
:1018500063F6E700B7070020238A07007D5723823D
:10186000E18C2383018CA382018C9387218C9A23A2
:101870007D179AA3924799EB31016FE01F8393057F
:10188000401F31457D2A2391A18C75BFEFF0AFD861
:10189000E5B7EFE2FF8081473DA0139717003306BD
:1018A000F700931616001386C186B29623900600A1
:1018B000239106003E9793161700B29623920600D6
:1018C000850793F7F70F2147E379F7FC2381018A16
:1018D000A381018A2397018A814709A81387418A36
:1018E0003E9723000700850793F7F70F2147E3771B
:1018F000F7FE814709A81387818B3E9723000700D5
:10190000850793F7F70F2147E377F7FEB707002026
:10191000238A07009305401F314525222391A18C7E
:101920002383018C938701859833A382E18C6FE038
:10193000CFF70323C5001841B707008093C7F7FF0F
:101940007D8F4C412D8F1045318F93161700B98E26
:1019500093571300B58FB3C767000CC150C11397DD
:10196000A700358F18C55CC5858B99C71C493D8E6E
:1019700050C15C493D8F18C5828058451C411445B3
:10198000A182B6973D8F858B99C31C4D3D8F3A85BB
:101990008280EFE2EFF02A840CC1B717708F938733
:1019A000E71E1CC95CC1B70779FC9387F7F15CC9D6
:1019B0001CC5B70794379387F7DF1CCD5CC58546F8
:1019C000A1A813F636009387F6FF8D8B8A07A2979E
:1019D0009C4313D7E701B98F1397C7003E97931520
:1019E0003700BE95139745001D8F93152700998DDD
:1019F000139725001D8F931537002E9793153700E9
:101A0000BE9513972500BA97B6971317260022970D
:101A10001043B18F1CC385069D47E3F4D7FA814478
:101A200021A02285393785049D47E3FC97FE6FE0AE
:101A3000CFE7EFE2EFE62A84ED3D22853D3F6FE000
:101A4000CFE6EFE2EFE52A84AE841385818CD537AB
:101A500093150501C18133858440EFE0AFE54181F5
:101A60002295420541816FE04FE403C7A18E89476B
:101A70006303F70082807DFD83C7C18EE5DF03C766
:101A8000B18E060793870185BA97D8230507D8A397
:101A9000D5B783C7A18E05476389E70413978701EC
:101AA000618709C70947638FE708828009C58547B1
:101AB0006302F502828083C7018585078D8B2388A9
:101AC000F184A382018E2383018E130700FC2382FD
:101AD000E18E8280138701851C3385079D8B1CB3A3
:101AE000130700FC2382E18E828009C58547630EBF
:101AF000F502828093870185B83383C6B18EB357D0
:101B0000D740858B99CB8547B397D70093C7F7FF0D
:101B10007D8F93870185B8B382808547B396D700C0
:101B2000558F93870185B8B382801387B18E1C23AC
:101B3000850793F7F70F1CA311476373F706A38577
:101B4000018E828009C585476306F504828003C73C
:101B5000C18E19CB03C7B18E060793870185BA974B
:101B6000D8230507D8A3828083C6B18E9D4763E240
:101B7000E70285069D8A93870185BC33B3D7D7409A
:101B8000858B89E705071377F70FCDB7A385D18E2E
:101B9000828082809387C18E98231337170098A381
:101BA0008280B707002083C7870713F7170061C338
:101BB0003707002013078707582B93761700C5CAED
:101BC00093F62700CDE693762700D5E203C601857C
:101BD0008D46630ED608EFE2AFCCB706002093E740
:101BE0008700238CF6069386860713678700D8AA9A
:101BF0001387A18E1C23850793F7F70F1CA30947B2
:101C00006387E70203C7A18E894763F4E700238552
:101C1000018E03C7A18E89476302F702EFF07FC7E9
:101C200003C7A18E85476301F7046FE00FC8938750
:101C30000185BC33E1FB2385018EE9B703C7B18E73
:101C400081469D47E3ECD7FC1D8B93870185BC3310
:101C5000B3D7E740858B91E70507850693F6F60F26
:101C6000CDB7A385E18E5DBFA385018E7DBF828048
:101C7000EFE20FC31385818CEFF0BFDB1D890144B8
:101C800021A005041374F40F9D4763E8870233070E
:101C9000A4001D8B93870185BC33B3D7E740858BA8
:101CA000EDD3B707002083C75701E38CE7FCB707E4
:101CB0000020A38AE700EFF0DFBDA1476305F40031
:101CC00005456FE08FBE0145EDBFEFE26FBD1385A7
:101CD000818CEFF01FD64205418193173500898F23
:101CE000139547001D8D93175500C1839387071ED9
:101CF00037070020231BF7006FE02FBBEFE24FBA3E
:101D000003C4018593870185943383C7A18E05475A
:101D10006389E70C13978701618711C709476382BD
:101D2000E70E6FE08FB8B707002003C75701914750
:101D3000E309F7FE83C7518E8DEB1387618E1C2359
:101D40008507858B1CA3939716000D67130787D80B
:101D5000BA979E238583A382F18E13878186230100
:101D60000700A3000700238401861387518E1C23DC
:101D7000FD1793F7F70F1CA30947636B870403C58F
:101D8000618E0DC586060D67130787D8BA969A220D
:101D90007D17638CE7021305F00F11476368F700A6
:101DA000B307F7403355F5401375F50F93878186D8
:101DB000A2979C23E387A7F6EFF00F909387818685
:101DC0003E9408A0EFF02F85A9BF1305000AF1B7D4
:101DD0002384018693878186A380070023810700DF
:101DE00089B793870185BC3303C7B18EB3D7E7406A
:101DF000858B91C71307F0072384E1861DB7014740
:101E0000E5BF83C7C18E99C39307F0072384F1868A
:101E100009BFB7070020938787079305200DCEA33E
:101E20006547FAA337260000130626BA90C7B726DF
:101E300000009386A6A6D4C737270000130727A95A
:101E400098CB8EAF239D0700D0CF94D3D8D3828078
:101E5000EFE20FA5311183C7418E99C7FD1793F7A4
:101E6000F70F2382F18EA9C783C4E18E958083D7B3
:101E7000818E99C7FD17C207C1832394F18E85CF48
:101E80001387E18E1C23850793F7F70F1CA303C765
:101E9000A18E85466305D72093168701E1868DC202
:101EA00089466308D728EFF07FE551016FE0EF9F87
:101EB000EFE08FFC55BF2385018EEFE0EFFBC9B744
:101EC000371701408546232AD740858BC1E3938786
:101ED0000185BC33E9DBB707002083D767018DC7D5
:101EE000B707002083C657019397260037070020C5
:101EF00013070700BA979C4381CB11476366D7004D
:101F000083C5E18E0145829783C7E18E8D8BC1FF2A
:101F100037070020130767011E23FD17C207C1837F
:101F20001EA34547E361F7F8EFE0FFEEB707002097
:101F300083D767014547638FE70621476378F70A30
:101F400041461D8E42064182814779A0EFE06FC174
:101F500042054181854763FBA702931715003E9513
:101F600093173500C207C183A183890703C7D18EA8
:101F700093160701C18263E8D70263FFF600E547C5
:101F800063ECE7000507A386E18E39A083C7D18EF5
:101F900081C7FD17A386F18E83C5D18E13058006F8
:101FA000EFE0AF9A2DB78947E3F8E7FE7D17A386E8
:101FB000E18EDDB7EFF0DFCBE31705EEEFF0FFD0FA
:101FC000DDB51307F00F3357C7405408BE9623887A
:101FD000E6FE850793F7F70F3D47E374F7FE3D46AE
:101FE0004C0013058006EFE0AF9A75BD1D47636B8B
:101FF000F704C5C713F67700814795A0139717001C
:102000003306F700931616001386C186B296239006
:102010000600239106003E9793161700B29623926E
:102020000600850793F7F70F2147E379F7FCB70719
:10203000002003C757019307F00FE316F7E6EFF010
:102040003FC395B58147CDB71307F00F3357C7404E
:102050005408BE962388E6FE850793F7F70F3D47A1
:10206000E374F7FE3D464C0013058006EFE04F9207
:102070001DBD58083E97FD562308D7FE850793F7E8
:10208000F70F3D47E377F7FE3D464C00130580060A
:10209000EFE00F90EFF07FC339B58147DDB79306CE
:1020A00000FC2382D18E8D83858B89CBB7170140AD
:1020B00003A7C7401347170023A6E7409305000472
:1020C00013058006EFE06F88EFE0FFD4014421A004
:1020D00005041374F40F9147E3E787DC22C09317DC
:1020E00024003707002013070700BA979C4381CBD1
:1020F00003C5B18E83C5E18E13650508829783C73A
:10210000B18EE39787FC93F71400F9D38245939738
:102110001500B386B700139716009386C1863697CD
:10212000414612A332A3AE9713971700369752A3D6
:1021300045B7930600FC2382D18E9583858B89CB8E
:10214000B717014003A7C7401347170023A6E7406E
:102150009305000413058006EFD03FFFEFE0BFCBEF
:1021600083C7C18E99E3014489A003C4B18EEFE017
:102170004F9F060493870185A297C8B3EDB79317C5
:102180001400B3868700139716009386C18636978E
:102190002310070023110700A29713971700369703
:1021A0002312070005041374F40F9147E3ED87CE63
:1021B00093870185BC3322C0B3D78740858BE1D399
:1021C000931724003707002013070700BA979C4392
:1021D00081CB03C5B18E83C5E18E13650508829757
:1021E00083C7B18EE39087FC93F71400C5DF824567
:1021F00093971500B386B700139716009386C18690
:1022000036971306000212A332A3AE971397170056
:10221000369752A341BF828001A01387018F1E23EE
:102220008507C207C1831EA31307F01F6379F70058
:102230002398018E9387418F9843050798C383D7CE
:10224000018F8D8B8DC3EFE0AF9B83D7018F858B83
:1022500091CF83D7018F858B89EFB7F700E023A259
:10226000070073002030EFE09FBBF1BFEFE0CF85A8
:10227000CDB7EFE0AF86D5B7B707002083A78702B9
:10228000A583FD1737F700E01CCB23240700BD47CB
:102290001CC323220700B7E700E0056723A0E7106F
:1022A0008280EFD2FFDF511123110100894426C241
:1022B000930780023EC4930700077C808A85371409
:1022C000014013050440792364808A851305048046
:1022D000512341473AC4914464808A8513050480A0
:1022E000952B85477C808A8513050440A523930799
:1022F00080023EC4930710087C808A853715014010
:10230000912B64808A8513050440A92399477C801A
:10231000F1473EC48A85371501402D2BA1475CC883
:10232000930700041CC841473AC4930780047C808B
:102330008A8537150140392B31016FD01FD7EFD275
:102340003FD60945EF00407B212A854537052010FF
:10235000EF00700B85450565130555A3EF00D00808
:10236000EFF03FF4EFE0EF82EFE00FCFB71701405F
:1023700088471375050213351500EFE06FA8EFD0FD
:102380001FE5EFE01FA0D12193870185EE27C98DBE
:102390001385818CEFF0EFDFEFF0BFA7EFF0DFEDFB
:1023A00019A0EFF0FFAA37F700E0832707D1DD9BE4
:1023B0002328F7D07300501083D7018F8D8BE5F75A
:1023C000CDB7B72702409843719B98C3984398C3F1
:1023D000B7170240D843D8C38280EFD27FCC3717DB
:1023E00002401C4F93E707021CCFB71701409386AA
:1023F000074003A707401377F7F023A0E74003A7A0
:1024000007401367070823A0E74089479CCAEFF0FD
:102410005FFB6FD09FC9EFD2BFC8B7170240984388
:102420001367170098C3D843B706FFFC758FD8C34E
:102430009843B706F7FEFD16758F98C39843B70605
:10244000FCFFFD16758F98C3D843C176FD16758FB6
:10245000D8C337079F0098C7EFF03FF86FD0FFC48D
:10246000B7170240DC43B18B11476385E70621476C
:10247000638BE70691CB37070020B7376E01938750
:1024800007602324F70209A837070020B7376E0139
:10249000938707602324F702B7160240DC4291833A
:1024A00013F7F700B707002093878701BA978C23AB
:1024B00093F5F50FDC4293F70708B9EFEFD25FBE53
:1024C00037040020130484020840EFD0BFC008C0C6
:1024D0006FD0BFBD37070020B7376E019387076005
:1024E0002324F70255BFB7170240DC431397F700C8
:1024F000634B070037070020B777DC02938707C0DC
:102500002324F70251BF37070020B777DC029387F7
:1025100007C02324F70249B7B70700209387870233
:102520009843B355B7008CC3828001A001A001A0DD
:1025300001A001A001A001A001A001A001A001A093
:1025400001A001A001A001A001A001A001A001A083
:1025500001A001A001A001A001A001A001A001A073
:1025600097E1FF1F9381012F138101FB17150000D5
:102570001305C58297E5FF1F9385C5A817E6FF1FC2
:10258000130646AD63FAC5008322050023A055005B
:1025900011059105E3EAC5FE17E5FF1F130585AB9D
:1025A0009385C18F6377B500232005001105E36D86
:1025B000B5FE93020008739002308D427390428002
:1025C00097E2FFFF938202A493E2320073905230AD
:1025D000EFF07FE4970200009382A2D6739012344A
:1025E00073002030B7270140938707406303F5004D
:1025F0008280EFD2FFAA854513050020252581455D
:102600001305002005256FD05FAA5C413707F1FF55
:102610001307F7EF7D8F9C41D441A206D58FD98F48
:102620005CC11C4537F7F1FF1307D77F7D8F9C49AD
:10263000D445D58F94458606D58FD98F1CC55C555A
:10264000370710FF7D177D8FDC29FD1793F7F70FF4
:10265000D207D98F5CD5828091C51C4593E71700BE
:102660001CC582801C45F99B1CC582801C4593E7D4
:1026700087001CC582801C45A18B99C305458280BB
:10268000014582801C4593E747001CC582801C459C
:10269000918B99C3054582800145828099C51C456F
:1026A00037075000D98F1CC582801C453707B0FF03
:1026B0007D17F98F1CC58280A54763F7B7040323F4
:1026C000C500138765FF93171700BA971D47331787
:1026D000F7001347F7FF33776700B396F600558F7F
:1026E00058C5994763E3C70458597D1693172600C8
:1026F0003E96FD47B397C70093C7F7FFF98FB39591
:10270000C500CD8F5CD98280032305011397150086
:102710002E979D47B397E70093C7F7FFB3F767007E
:10272000B396E600D58F1CC96DBFB14763E2C702FF
:1027300018596516931726003E96FD47B397C700B4
:1027400093C7F7FFF98FB395C500CD8F1CD9828051
:1027500054554D16131726003A96FD47B397C700F8
:1027600093C7F7FFF58FB395C500DD8D4CD58280FB
:10277000684542054181828091C55C4193E70740ED
:102780005CC182805C4193F7F7BF5CC18280A54742
:1027900063FDB7040323C500138765FF9317170074
:1027A000BA971D473317F7001347F7FF33776700D2
:1027B000B396F600558F58C5145D93D746018D8B9F
:1027C000B307F64093F7F70F890793F7F70F1397BF
:1027D0002700BA977D473317F7001347F7FF758F28
:1027E000B395F5004D8F18DD828003230501139703
:1027F00015002E979D47B397E70093C7F7FFB3F7F0
:102800006700B396E600D58F1CC97DB7711102C071
:102810002AC08247BE95938585022EC08247884391
:1028200042054181110182801C41FD8D99C1054500
:102830008280014582805C41370700FA7D17F98F5D
:102840005CC15C41DD8D4CC18280B7F7FF1F03A5E1
:10285000477C82809C4513F6F700C18B99C3DC410D
:102860005D8E9C21B9CB03230500014719A05CC9EB
:1028700005079D4763E1E7048547B397E700962185
:10288000FD8EE397D7FE93122700BD46B396560000
:1028900093C6F6FFB3F66600331356003363D300D6
:1028A000944593028002E38456FC93028004E391F2
:1028B00056FC1CC975BF232065009A219307F00FB1
:1028C00063F2E70603234500014721A05CC989A004
:1028D00005079D4763E6E704930787008546B3979E
:1028E000F6009621FD8EE395D7FE93122700BD4694
:1028F000B396560093C6F6FFB3F666003313560040
:102900003363D30083A2850093068002E380D2FC68
:1029100083A2850093068004E39CD2FA1CC94DBFB4
:10292000232265008280EFD2AFF711112A84AE8492
:102930004A2142054181137505FC93170501C183A6
:102940003EC02800F922C247B7450F0093850524F1
:102950003EC23E85EFD00FF8420541810247598DB6
:102960004AA01E20C207C183F99BC207C1831EA0D3
:102970008C40E1679387076A63EDB70086051245CF
:10298000EFD04FF5420541818D4763E0A704114523
:102990002DA8FA20B167FD17630FF7049397150070
:1029A000AE9713973700BA951245EFD0AFF24205B4
:1029B000418191675D8D8567FD17E98F99E3136507
:1029C0001500E1775D8D420541814AAC1E2093E7F9
:1029D00017001EA01E20C207C18393F757BFDA203D
:1029E000B624558FD98F1EA0DE249A24D98F1EA419
:1029F00071016FD08FEB93971500BE951245EFD004
:102A00006FED4205418145BF91C51E2193E7170037
:102A10001EA182801E21C207C183F99BC207C18308
:102A20001EA1828091C51E2193E707101EA18280FE
:102A30001E21C207C18393F7F7EFC207C1831EA10E
:102A4000828091C51E2193E707201EA182801E214E
:102A5000C207C18393F7F7DFC207C1831EA182803B
:102A600091C51E2193E707401EA182801E21C20747
:102A7000C18393F7F7BFC207C1831EA182800EA94D
:102A800082800A291375F50F828019C693E5150017
:102A9000C205C1810EA9828093F5E50FD5BF5A29E1
:102AA0001E2DC207D98F370700017D17F98FED8FD3
:102AB0006384B7000145828005458280611102C2AE
:102AC00002C02AC093D7C5013EC2B7070001FD1757
:102AD000FD8D924799CB8247D1073EC082479C43E8
:102AE000FD8D89C9054521018280C1818247E107A9
:102AF0003EC0EDB70145C5BF23ACA18E8280B7169D
:102B00000240DC4241771307F77FF98F5D8DC8C221
:102B10008280EFD2EFD82A84B7170240DC43B18B12
:102B200011476385E70821476388E70899C7B737E6
:102B30006E01938707601CC131A0B7376E01938780
:102B400007601CC1B7160240DC42918313F7F700FF
:102B5000B707002093870704BA978C2393F5F50FE6
:102B6000DC4293F70708A5EF0840EFD0AFD648C086
:102B7000484008C448C4B7170240DC43AD83FD8B0E
:102B800013D737008A07F18B5D8F937637018D4716
:102B900063F3D7005117B70700209387C702BA978E
:102BA0008C23EFD02FD308C86FD02FD0B7376E014A
:102BB000938707601CC179B7B7170240DC431397AE
:102BC000F70063480700B777DC02938707C01CC192
:102BD00095BFB777DC02938707C01CC1A5B71C401F
:102BE000B3D5B7004CC069B799C5371702401C4F21
:102BF0005D8D08CF8280371702401C4F1345F5FFCB
:102C00007D8D08CF828099C5371702405C4F5D8D5E
:102C100048CF8280371702405C4F1345F5FF7D8D0A
:102C200048CF828099C5371702405C475D8D48C701
:102C30008280371702405C471345F5FF7D8D48C7FA
:102C4000828000000000000000010101010101017B
:102C50000101020202020202020202030303030351
:102C6000030303040404040404050505050506061E
:102C700006060607070707080808080909090A0AD7
:102C80000A0A0B0B0B0C0C0C0D0D0D0E0E0F0F0F7B
:102C90001010111111121213131414151516161702
:102CA00017181819191A1A1B1C1C1D1D1E1F1F206E
:102CB000202122222324252526272728292A2B2BB9
:102CC0002C2D2E2F2F3031323334353636373839DC
:102CD0003A3B3C3D3E3F4041424344464748494AD7
:102CE0004B4C4D4F50515253555657585A5B5C5EA2
:102CF0005F606263646667696A6C6D6E707173743D
:102D00007678797B7C7E8081838486888A8B8D8FA0
:102D100091929496989A9B9D9FA1A3A5A7A9ABADCC
:102D2000AFB1B3B5B7B9BBBDBFC1C4C6C8CACCCFBC
:102D3000D1D3D6D8DADCDFE1E4E6E8EBEDF0F2F56A
:102D4000F7FAFCFF04140111070A1A0D1D00000018
:102D50000000000012345501230123440123012304
:102D60004412340000022222432104321043210481
:102D7000432143210432102222220000FFF0F00000
:102D8000F000FF1004000000FF00BF007F005500AE
:082D90004400290022001D008F
:102D9800C40E000020100000CC13000074120000C4
:102DA80032150000FFFF09000102030405060708A9
:102DB800010203040506070800366E01020406082E
:102DC80004080C10081018201020304020406080A3
:102DD80001020304050607080102030405060708A3
:00000001FF
